:060000000A128A110E280D
:10000800FE000308F1000408F2000A08F3000A12CF
:100018008A11BC2D0A128A11852FF42A82233208EC
:10002800770603191C287708B2001230F9003C281B
:100038000A30F40076082F230A128A11C1000A3008
:10004800F40076084B230A128A11C2000A30F40021
:1000580077082F230A128A11C3000A30F4007708A0
:100068004B230A128A11C4006430AF00AE01AE0AF5
:100078002B08031908003008760603190800093010
:100088007602031C0800163076020318080076086A
:10009800B000AE01AE0AB501B50AFF30BC008F3022
:1000A800BD000130BC020030031CBD03BD023C0A88
:1000B80003193D0A031D5528B5010800822331089C
:1000C800023A0319F60A183076020318F6013108C5
:1000D800033A0319F603FB307602031C7528173020
:1000E800F6000A30F40076082F230A128A11C1009C
:1000F8000A30F40076084B23C2000A30C300C4005B
:10010800080082233108023A031D8C28F70AA3014C
:100118003C3077020318F7013108033A031D96288B
:10012800F703A301FB307702031C9C283B30F70040
:100138000A30C100C200F40077082F230A128A117E
:10014800C3000A30F40077084B23C4000800822358
:100158003108023A0319A10A183021020318A10133
:100168003108033A0319A103FB302102031CBE28FE
:100178001730A1000A30F40021082F230A128A112F
:10018800C1000A30F40021084B23C2000A30C30022
:10019800C400AE01AE0A080082233108023A0319EE
:1001A800A20A3C3022020318A2013108033A0319BB
:1001B800A203FB302202031CE3283B30A2000A30D2
:1001C800C100C200F40022082F230A128A11C300BA
:1001D8000A30F40022084B230A128A11CC28822301
:1001E8003108023A0319F50A08307502031CFE2883
:1001F800F501F50A3108033A0319F503F508031D5B
:1002080007290730F500C1010A30C200C30075088C
:10021800C400AE01B108031908000E290230822378
:100228003102031C1E29240803191C29A4011E29B4
:10023800A401A40AC101C10A0A30C200C3002408EB
:10024800C400B108031908002529023082233102AD
:10025800031C3529250803193329A5013529A501CA
:10026800A50A0230C1000A30C200C3002508C40034
:10027800B108031908003C29023082233102031C0B
:100288004C29260803194A29A6014C29A601A60AC1
:100298000330C1000A30C200C3002608C400B108F8
:1002A800031908005329023082233102031C6329F1
:1002B800270803196129A7016329A701A70A0430A0
:1002C800C1000A30C200C3002708C400B1080319DE
:1002D80008006A29023082233102031C7A2928087F
:1002E80003197829A8017A29A801A80A0530C100AC
:1002F8000A30C200C3002808C400B1080319080066
:100308008129023082233102031C9129290803190B
:100318008F29A9019129A901A90A0630C1000A302B
:10032800C200C3002908C400B108031908009829AD
:10033800023082233102031CA8292A080319A6299E
:10034800AA01A829AA01AA0A0730C1000A30C200D6
:10035800C3002A08C400B10803190800AF29822382
:100368003108023A0319A00A15302002031CBE29DD
:100378001430A0003108033A0319A003FB3020020F
:100388000318A0010830C1000A30C200F400200898
:100398002F230A128A11C3000A30F40020084B23C5
:1003A8000A128A11C40020082D3E9500B1080319CD
:1003B8000800DA29023082233102031CEA292B08BB
:1003C8000319E829AB01EA29AB01AB0A0930C100DE
:1003D8000A30C200C3002B08C400B1080319080082
:1003E800F129023082233102031C012A2C08031947
:1003F800FF29AC01012AAC01AC0AC101C10AC20142
:100408000A30C3002C08C400B10803190800082AE0
:1004180082233108023A0319C50A08304502031835
:10042800C5013108033A0319C50309304502031C05
:100438001F2A0730C500450867230A128A11C1011F
:10044800C10AC201C20A0A30C3004508C400B10883
:10045800031908002B2A0A30F40076082F230A1201
:100468008A11C1000A30F40076084B230A128A1157
:10047800C2000A30F40077082F230A128A11C30039
:100488000A30F40077084B230A128A11C400B10815
:10049800031D4B2A3C30B300F90108008223AE014A
:1004A800AE0ABE010A303E020318672A3E08C100A0
:1004B80076230A128A117C230A128A1103193D0A2B
:1004C8000319562A5F2A0A30F40076082F230A12E5
:1004D8008A11C100BE010A303E020318802A3E0874
:1004E800C20076230A128A117C230A128A11031980
:1004F8003D0A03196F2A782A0A30F40076084B233C
:100508000A128A11C200BE010A303E020318992A53
:100518003E08C30076230A128A117C230A128A1124
:1005280003193D0A0319882A912A0A30F40077082A
:100538002F230A128A11C300BE010A303E02031893
:10054800B22A3E08C40076230A128A117C230A12B2
:100558008A1103193D0A0319A12AAA2A0A30F400AC
:1005680077084B230A128A11C400831603178C18C4
:10057800B92A0C3083128D0076080A128A11752761
:100588000A128A1103188B178C18C82A0D30831287
:100598008D0077080A128A1175270A128A11031822
:1005A8008B178C18D52A0E3083128D00031323085D
:1005B80003170A128A1175270A128A1103188B1752
:1005C80082232C080319502AC50A08304502031C47
:1005D800EF2AC501C50A450867230A128A11502A5D
:1005E8007908003A03191228013A03196228033AD4
:1005F80003198528013A0319AB28073A0319D028AB
:10060800013A0319F328033A03191229013A031985
:1006180029290F3A03194029013A03195729033A9E
:1006280003196E29013A03198529073A03199C29E8
:10063800013A0319B329033A0319DE29013A0319C8
:10064800F5291F3A03190C2A013A03192F2A033AEC
:10065800031D0800522A8223B800BA01740803193E
:10066800492BB901B90AF41B3C2B0310F40D362BA6
:100678000310BA0D74083802031C462B7408B8021C
:100688003A140310F40CB90B3C2B3A080800B900D3
:100698000830BA00BB013908B80007300310B80C9D
:1006A800FF3E0310031D532B3B0D3804BB00031002
:1006B800B90D74083B02031C632B7408BB02BA0B08
:1006C8004F2B3B080800B8001F3086053808F40097
:1006D80004300310F40DFF3E0310031D6E2B740D40
:1006E80086040800BE0AFF30BC000F30BD000800B9
:1006F8000130BC02031CBD033C0A0800831203132B
:10070800080083160F178F160F128B018C018D01AD
:1007180083128C018D018501860187018901831669
:1007280003178801890120300313850007308600EC
:1007380087010830890083128501860187018901B4
:1007480007308316810081130730950083129001CA
:10075800920197019D0194010B17831681120111D3
:10076800811401148111831281018B160B119015CC
:100778001015901480308F00101483160C1441301B
:1007880092000130831295000C3097007C30920063
:1007980003178D013F3083168C050C1483120C0847
:1007A8000313A100013003178D003F3083168C0519
:1007B8000C1483120C080313A200023003178D00D7
:1007C8003F3083168C050C1483120C080313A40005
:1007D800033003178D003F3083168C050C148312E9
:1007E8000C080313A500043003178D003F3083164F
:1007F8008C050C1483120C080313A600053003178C
:100808008D003F3083168C050C1483120C080313DB
:10081800A700063003178D003F3083168C050C1493
:1008280083120C080313A800073003178D003F300C
:1008380083168C050C1483120C080313A9000830C6
:1008480003178D003F3083168C050C1483120C0897
:100858000313AA00093003178D003F3083168C0557
:100868000C1483120C080313A0000A3003178D0020
:100878003F3083168C050C1483120C080313AB004D
:100888000B3003178D003F3083168C050C14831230
:100898000C080313AC000C3003178D003F3083168F
:1008A8008C050C1483120C08F6000D308D003F30B7
:1008B80083168C050C1483120C08F7000E308D007B
:1008C8003F3083168C050C1483120C080313A30005
:1008D80018302102031C722C0730A1003C30220280
:1008E800031C782C0F30A20002302402031C7E2C3B
:1008F800A401A40A02302502031C842CA401A40A22
:1009080002302602031C8A2CA401A40A0230270202
:10091800031C902CA401A40A02302802031C962C64
:10092800A401A40A023029020318A40102302A02F1
:100938000318A40115302002031CA42C1430A000B5
:1009480002302B02031CAA2CAB01AB0A02302C028A
:10095800031CB02CAC01AC0A19307602031CB62C6F
:100968000C30F6003C307702031CBC2C2230F70018
:100978003C3023020318A30120082D3E95000730C0
:100988000A128A1167230A128A118B17851AD12C29
:10099800B701B70AB601B60AD22CB701B708031DCA
:1009A800CA2C36080319F62C83160F178F160F1248
:1009B8002030850007308600870183128501860173
:1009C80087018901831681139500831245080A124D
:1009D8008A1167230A128A118B1612150C30970098
:1009E800B601F901330823060319132D2308B300B0
:1009F8003408031DB403340B072DF9010A128A11B8
:100A0800D9260A128A11790803190E2D7908123A83
:100A1800031D132D0A128A1111200A128A1183123A
:100A28000313310B342DB508031D342DF90A0A12AE
:100A38008A1111200A128A1183120313B108031DA7
:100A4800202DFF30BF001F30C0000130BF02031C43
:100A5800C0033F0A0319400A031D292D0F30B400B3
:100A680002303102031C562DB508031D562D790896
:100A78000319562D0A128A1111200A128A11FF3001
:100A880083120313BF001F30C0000130BF020030C3
:100A9800031CC003C0023F0A0319400A031D492D65
:100AA8000F30B400310803196E2D350803196E2D67
:100AB800B501B108031D5D2DFF30BF00C000013036
:100AC800BF020030031CC003C0023F0A0319400ADA
:100AD800031D632D76082106031DB62D770822060F
:100AE800031DB62DA308031DB62D24080319802D58
:100AF800750B802DB501B50A25080319892D7508D0
:100B0800023A031D892DB501B50A26080319922D4D
:100B18007508033A031D922DB501B50A2708031974
:100B28009B2D7508043A031D9B2DB501B50A2808AD
:100B38000319A42D7508053A031DA42DB501B50A9E
:100B480029080319AD2D7508063A031DAD2DB50109
:100B5800B50A2A080319B62D7508073A031DB62DDC
:100B6800B501B50A770822060319CA2CB501CA2CA3
:100B780001300B1D00398B1E003900380319E62D92
:100B880036260A128A11AF032F0BCE2DF908031D42
:100B9800CE2DAE012E080319D52D35080319D52DF4
:100BA8008515B50803198511B1018618DD2DB10128
:100BB800B10A0618E12D0230B1000619E52D0330FF
:100BC800B1000B110130D6260C1C003983160C1C01
:100BD8000039003803192D2E803083128F00A30AA4
:100BE8003C302302031CFA2DA301F70A3C3077029C
:100BF800031C002EF701F60A18307602031C072E94
:100C0800F601F50AAD0A08307502031C0D2EF50130
:100C1800F50A10302D02031C142E950197010D2E94
:100C2800370803192B2E121197018B128316950181
:100C38008117850186018701831285018601870155
:100C480083160F138F120F1263000000851683128C
:100C58000C1073088A007208840071088300FE0E65
:100C68007E0E0900F80A043078020318F801D62627
:100C780087130713871207124630F000F003700835
:100C8800FF3A0319772E422ED62605145F2ED62654
:100C980005145B2ED626051006126A2ED6260510D8
:100CA800732ED62605100616602ED62605100612B7
:100CB800652ED6260510061286116B2ED62605102F
:100CC80006168611752ED626051006168615851069
:100CD8009D2ED62605100612742ED6260514061645
:100CE800861585149D2E7808413E840083130008DC
:100CF800003A0319482E013A03194B2E033A0319F7
:100D08004E2E013A0319522E073A0319552E013A6D
:100D18000319592E033A03195D2E013A0319622E5D
:100D28000F3A0319672E013A03196D2E033A031976
:100D3800712EF808031DA92E7808413E84000A3058
:100D480000020318A92ED6268717780BB42E780828
:100D5800413E84000A3000020318B42ED626071735
:100D68007808023A031DC12E7808413E84000A30F3
:100D780000020318C12ED62687167808033A031DE9
:100D8800CE2E7808413E84000A3000020318CE2E89
:100D9800D6260716D6262E080319D42E871508003E
:100DA80087110800831203130800831603178C1891
:100DB800D92E83128D0103132108031775270A12F0
:100DC8008A1103188B178C18E72E013083128D00B7
:100DD80003132208031775270A128A1103188B17A1
:100DE8008C18F42E023083128D0003132408031785
:100DF80075270A128A1103188B178C18012F0330D4
:100E080083128D0003132508031775270A128A1108
:100E180003188B178C180E2F043083128D000313C0
:100E28002608031775270A128A1103188B178C18BE
:100E38001B2F053083128D0003132708031775270E
:100E48000A128A1103188B178C18282F0630831260
:100E58008D0003132808031775270A128A1103182F
:100E68008B178C18352F073083128D000313290830
:100E7800031775270A128A1103188B178C18422F2B
:100E8800083083128D0003132A08031775270A12E6
:100E98008A1103188B178C184F2F093083128D0075
:100EA80003132008031775270A128A1103188B17D2
:100EB8008C185C2F0A3083128D0003132B0803173C
:100EC80075270A128A1103188B178C18692F0B3093
:100ED80083128D0003132C080317752703188B172B
:100EE80008008C003F3083168C0503108B1B0314FD
:100EF8008B130C1555308D00AA308D008C140C11F5
:100F08000800F801F901AD01AE01AF01B001B1016E
:100F1800B201B301B401B501B601B7010130C10096
:100F28000230C2000330C3000430C4000630C500DC
:100F38000130F5000C30F6002230F70083010A1268
:040F48008A11852B5A
:04400E00C424FF3E89
:1042000007000F0001000100010001000100000093
:1042100000000A00010001000C0022000000FF0065
:00000001FF
